:10000000600400204909000045090000450900007E
:1000100000000000000000000000000000000000E0
:100020000000000000000000000000004509000082
:100030000000000000000000450900004509000024
:10004000450900004509000045090000E9060000D7
:1000500049030000450900004509000000000000B8
:1000600045090000450900004509000000000000A6
:100070000000000045090000450900004509000096
:100080000000000000000000450900000448054B86
:1000900010B5834203D0044B002B00D0984710BD0D
:1000A000580C0000580C00000000000006480749EA
:1000B000091A8B10C90FC91810B5491003D0044B89
:1000C000002B00D0984710BD580C0000580C0000C1
:1000D0000000000010B5074C2378002B09D1FFF772
:1000E000D5FF054B002B02D0044800E000BF0123E0
:1000F000237010BD0000002000000000580C00001C
:10010000054B10B5002B03D00449054800E000BFA3
:10011000FFF7CCFF10BDC046000000000400002027
:10012000580C00000122014BC25470471B000020F4
:10013000F0B5C0238026802580240E4A0E49DB05B9
:10014000F6015E600D4891620D49AD0091625D60FF
:1001500090620C48640091625C60906220200A4FBB
:1001600091625860976291625E615D615C61586105
:10017000F0BDC04600440041004002400002024081
:10018000000002C00001024020000240F7B5012635
:100190001F27310083B2C2B238408140C020802581
:1001A0005209D201C0051418ED0588B22843104D3C
:1001B000A16052199062080C8446C02065461B0A53
:1001C000000605431F409562BE408025C022B7B29D
:1001D000ED053D435B09064FDB01D2059A18DB199B
:1001E00096609D62350C28439862A1615661F7BD07
:1001F0000044004110B50024094B9847094BE35CCB
:10020000002B08D0084B6200D15C9B185878074B34
:1002100000020843984701340C2CEDD110BDC046B4
:10022000310100001C0000205C0B00008D0100006B
:10023000024B034A5A6005221A60704710E000E042
:10024000FFFFFF0070B580250B0E0C4A0C4CD8B296
:100250006D020138C0B2FF280AD118061B1A5918BE
:10026000802351605B02916011681942FCD070BD1F
:100270005460946016682E42FCD0EAE710E000E07B
:10028000FFFFFF0010B5041E03D00068431E984115
:10029000C0B24F220B4B0C49984723681A78D209F9
:1002A0000DD11A789207D00F002A08DB04211A78A2
:1002B0008A431A705A780B318A435A7010BD112044
:1002C0004042FBE7B5050000740B0000024A53787A
:1002D000DB09FCD17047C04600180040F8B5154C4A
:1002E000154D0700A847A84723789B0703D500238F
:1002F0002370A847A847012300262370A847A847D2
:100300000223A67066606661A6612278134323709B
:10031000A847102309490A4ACB67BFF34F8FBFF3A1
:100320006F8FC021490053501360064B30001F608F
:10033000F8BDC04600180040CD02000004E100E016
:1003400000E100E028000020F0B5274D85B02B69C2
:10035000EA68264E13400393039B30682B61431ECB
:100360009841C122224B2349C0B2984701235B42E6
:100370000093039B002B01D105B0F0BD03981E4FE5
:10038000B847013844B2631C06D12B69EA681340B0
:100390000393039B2B61ECE7184B012000229C4642
:1003A00083185B10D9B201916146DB005B5CA3420C
:1003B0000BD133680F2098470F2300930122A240EE
:1003C000039B934303930398DAE70199A34207DA67
:1003D0000131CAB28242E3D9009B0133E9D1EDE792
:1003E0000139C8B2F6E7C0460018004028000020D6
:1003F000B5050000890B0000C50A0000300C0000A4
:10040000F7B50568002D02D1114B9847F7BD0126BD
:100410002C0000278B680093B31A0193A6686368C9
:10042000B44693420DD863449B1A009E9E420CD959
:1004300023682700002B02D13800064BE5E71C009B
:10044000ECE7019EF3186344EFE7A542DCD0F3E745
:100450004506000071060000F8B50669037E013606
:10046000040045690661DB0702D4037E9B0717D5AC
:100470000223227E13432376F8BD270014370C4B4A
:10048000380098472B7C012B05D132002900380019
:10049000084B6E60984767692800EB6898473D00F5
:1004A000002DE9D06B68AA68F31A9342E5D2E3E71E
:1004B000790600000104000070B50D002B00040057
:1004C0005A1E9341421E904106493B221840064B5A
:1004D000984729002000054B98470020044B2061D5
:1004E000236070BD9E0B0000B50500009106000062
:1004F0005904000010B5024B1860024B984710BD1C
:100500002C00002031020000044B10B51C68044B85
:1005100098470100034B2000984710BD2C00002095
:10052000AD050000450200000D4B0E48196A1A6A1D
:100530000140920F92070A430B490A431A620222B2
:1005400099690A431F219A611A7F0A401A77082283
:10055000D9681142FCD08022196A0A431A62704796
:10056000000800400000FF0F020300000221024AC1
:1005700093698B439361704700080040064B10B5A8
:100580005A685A60054B9847054B9847054B984762
:100590003F20054B984710BD00400041BD050000BD
:1005A000290500006D050000DD050000FA239B0011
:1005B00058437047002800D100BE7047064B1A7A96
:1005C000D2B21A725A7AD2B25A729A7AD2B29A7253
:1005D000DA7AD2B2DA72704700040040C00709D557
:1005E0008023054A5B00936083235B02536053784A
:1005F000DB09FCD17047C046000C0040084B10B529
:100600009847084B98470124E0B2074B9847074B9F
:1006100098470120064B98470D2CF4D00134F3E79E
:10062000E50900003101000025010000F50100008E
:10063000090500000068002800D170478842F9D100
:100640000120FAE770B5074B0D000400984701231D
:10065000584039220449054BC0B2984723682B60A3
:10066000256070BD35060000B50B0000B505000023
:1006700003680B600160704703000068002801D028
:1006800002681A607047837ADB09FCD1704700006A
:10069000F8B50500431E98410C00012730220D4992
:1006A0000D4BC0B298470D4EEC6020002780B0473C
:1006B0002000B047802320002380B047A369802317
:1006C000DB002000A361B047054B0020E7711D60EF
:1006D000F8BDC046D30B0000B5050000870600003A
:1006E000300000200020704770B50125064B1C68C3
:1006F000E3681B7A2B4206D02368002B01D0200030
:100700009847E3681D7270BD30000020C02310229E
:10071000DB055A60094A0A4B11009362C0231B068D
:10072000936201220F2044310B7813430B70034B6B
:100730003233197881430A431A70704700440041EC
:10074000100000408023044A5B00116A0B431362CF
:10075000024B034A5A80704700040040000C0040DE
:100760001340000010B5054B9847054B98470022F1
:1007700004480549054B984710BDC0464507000091
:100780000D0700003400002000200042C1080000D6
:10079000104B114A10B55A80C0238022DB0512028B
:1007A0005A600E4A0E4B042193620E4B9362130063
:1007B0004F331A788A431A70012219780A430F219D
:1007C0001A70064B37331A780A401A70064B98474E
:1007D00010BDC046000C0040054000000044004130
:1007E00000800240000002C02109000010B502484C
:1007F000024B984710BDC04610E000E0F504000031
:100800001023044A91690B439361034B034A5A80B6
:100810007047C04600040040000C00400340000048
:1008200010B5074B9847482201200649064B9847C8
:100830000648074B04300360064B984710BDC0467E
:1008400001080000E80B0000B5050000340000209E
:10085000001000408502000010B50D4B98470D4B6D
:1008600098470D4B98470D4B984720230C4A9169A8
:100870000B4393610B4A0C4B5A800C4B98470C4B23
:1008800002000C4918000C4B98470C4B984710BDC0
:100890007D0500006507000091070000ED070000DE
:1008A0000004004004400000000C0040E506000089
:1008B0003C00002000140040B904000021080000A2
:1008C00070B50D002B0004005A1E9341421E90414A
:1008D000044939221840044B984729002000034B53
:1008E000984770BD010C0000B5050000990A000092
:1008F000012270B51500094C61680023D3185B1004
:1009000005D1814204D12368002B00D0984770BDE7
:100910002B008142F2D3FF22EFE7C04658000020AF
:100920000122054B524210B55A6000221A6003485A
:10093000034B984710BDC04658000020F108000046
:10094000DD020000FEE700001A4A1B4B10B51B49F0
:100950009A422AD100211A4B1A4A934228D3FF22E5
:10096000194B30219343194A93600222184B5A6263
:10097000184B987B88431039014399730C21987B5D
:1009800088430439014303209973997B81430A43C7
:100990009A738023104A51680B4353600F4B98475A
:1009A0000F4B9847FEE701CA01C38B42FBD3D1E747
:1009B00002C3D2E7580C0000000000200000002015
:1009C00000000020600000200000000000ED00E0BA
:1009D000FC7000410048004100400041150B000040
:1009E000FD05000010B5014B984710BD59080000E7
:1009F000437EDB09FCD17047F8B5214B0400C018D9
:100A00004342584194221F491F4BC0B29847E022ED
:100A10001E4BD2001B6820005D0115405A011C4B83
:100A20001C4E1B68DB0E1343DBB21D43B04723781B
:100A30009B0703D5002320002370B047012320002B
:100A40002370B04723002585022700252A336770CD
:100A50002000A570E5702575A584E5841D70A5802E
:100A6000B04720002561B04720002572B047200024
:100A7000A583B04725842000B0472770F8BDC04645
:100A800000E0FFBD1B0C0000B505000024608000E5
:100A900020608000F109000070B50500431E9841F8
:100AA0000C00C5220449054BC0B2984720002C60B9
:100AB000034B9847002070BD1B0C0000B5050000DB
:100AC000F909000010B5002802D000F003F8013049
:100AD00010BDC046414208401C2101231B0498421E
:100AE00001D3000C10391B0A984201D3000A0839BF
:100AF0001B09984201D30009043902A2105C401A74
:100B00007047C0461B1C1D1D1E1E1E1E1F1F1F1FC3
:100B10001F1F1F1F70B500260C4C0D4D641BA41029
:100B2000A64209D1002600F087F80A4C0A4D641B42
:100B3000A410A64205D170BDB300EB58984701360A
:100B4000EEE7B300EB5898470136F2E7440C00009B
:100B5000440C0000480C0000440C00000509090585
:100B60000E05050E090E0E09080909080E08080EE3
:100B7000080505082E2E2F68706C2F7764742F6877
:100B8000706C5F7764742E63002E2E2F68706C2F4C
:100B90006569632F68706C5F6569632E63002E2E34
:100BA0002F68616C2F7372632F68616C5F74696D5D
:100BB00065722E63002E2E2F68616C2F7574696C20
:100BC000732F7372632F7574696C735F6C697374C0
:100BD0002E63002E2E2F68706C2F7274632F687036
:100BE0006C5F7274632E63002E2E2F68616C2F6908
:100BF0006E636C7564652F68616C5F7764742E68D2
:100C0000002E2E2F68616C2F7372632F68616C5FEA
:100C10006164635F73796E632E63002E2E2F68709C
:100C20006C2F6164632F68706C5F6164632E630076
:100C3000010000000F000000F8B5C046F8BC08BC79
:100C40009E46704701010000F8B5C046F8BC08BCDC
:080C50009E467047D50000002C
:00000001FF
